:020000040000FA
:020000002928AD
:08000800F0000308F10083126F
:100010000B190C280C1324280B11F30A031D242898
:100020007214A00B1628F2150130A000AD0B1C288D
:100030000230AD000230F2067215AE0A2E08783A90
:10004000031D24287211AE0371088300F00E700E98
:100050000900850107309900831660308F008316F0
:1000600034309F008316FC308500831600308100F9
:100070008312203084008001840A841F3B284F2192
:10008000003058215C21E820B300B600013058212F
:100090005C21E820B200B500023058215C21E82044
:1000A000B100B4000230AD000130A00083160C177F
:1000B00083120C130B178B168B1708303F21AF20C0
:1000C0002108A200A300A400A500A600A700A80084
:1000D000A900051EFD28721C6B287210AA20F21DB3
:1000E0006B28F211AF20C72076206B28360821023A
:1000F000031883283508210203188B2834082102AD
:1001000003189828A2283303B6002F10AF1030141C
:10011000B014AE0108003308B6003203B5002F104A
:10012000AF143010B010851EAE01721DAF10080064
:100130003208B5003103B4002F14AF103010B010E6
:10014000AE0108003108B4002F10AF103014B01009
:10015000AE0108002F08F2183004850008000930AD
:100160009F0085010830FF3E031DB3288B139F14A9
:1001700063000000AA201E08831603109E1B013E88
:100180000318FF3E8312A1000C138B1708002A08E6
:10019000223E840021088000AA0A2A08083C03198C
:1001A000AA0022308400AB01AC010008AB070318A1
:1001B000AC0A840A04082A3C031DD528AC0CAB0CFD
:1001C000AC0CAB0CAC0C2B0C0318013EA1000800CE
:1001D000BB00BA01B9010830BC000310BA0DB90D5B
:1001E000BB0D031CF9283808BA070318B90A3708E9
:1001F000B907BC0BED28390808008B12051EFE2834
:100200000C30B700AF20C720B70B2108B700403033
:10021000B8000310B70CB80C031C0A2946218B1632
:10022000370C25210830BC000310B81B0314B80D8F
:100230002521BC0B14291D2110292F14AF143010B7
:10024000B010AA2019303F21372903182F292F1465
:10025000AF103010B010AA2004303F2137292F10E2
:10026000AF143010B010AA2004303F2137292F10CE
:10027000AF103010B010AA2008303F210800721CC7
:100280003F297210FF3E031D3F290800033058210B
:1002900037086121043058213808612108000330F3
:1002A00058215C21B700043058215C21B8000800B7
:1002B00083169B008312080083161C141A088312ED
:1002C000080083169A0083168B131C1555309D0069
:1002D000AA309D009C149C186B2983128B17080070
:02400E00E43894
:0A420000BF00A7009D0001000000B0
:10424000563431342E34303435342C342034313437
:104250003234203456346F346C3474342034413466
:10426000753474346F346D346F3474346934763427
:1042700065342034423461347434743465347234B7
:104280007934203456346F346C3474346134673488
:10429000653420344D346F346E34693474346F3483
:1042A00072342C34203450346934633470347234B2
:1042B0006F346A346534633474347334203428348E
:1042C00063342934203432343034313431342C34B2
:1042D00020345034653474346534203447347234B7
:1042E0006934663466346934743468347334203421
:00000001FF
